:020000020000FC
:10000000E8C009C01CC02FC04DC04DC04DC04EC07F
:10001000BFC0DEC04AC01F931FB71F932F9211E0CD
:100020002090A500210E2092A5001091A4001F1D74
:100030001093A4002F901F911FBF1F9118951F931D
:100040001FB71F932F9211E02090A700210E20923E
:10005000A7001091A6001F1D1093A6002F901F91BE
:100060001FBF1F9118951F922F923F924F921F937F
:100070001FB71F9310907300209072003CB44DB4D2
:100080003092730040927200311842083092A300FF
:100090004092A2001F911FBF1F914F903F902F9041
:1000A0001F90189518951895189518952F933F93AC
:1000B0000F92AF93BF93EF93FF931F922F923F92B4
:1000C0001F931FB71F9320E61BB114FB76F910FB9B
:1000D0002EF01CB1312E77FB36F011C01CB1312E41
:1000E0001AB111FB66F010906F00112009F442C0A4
:1000F00010906B0020906C00121834F132C01091F7
:100100009F001F71232C269426942694211A31F0E7
:10011000F0926F00F0926B0078682CC07068777F67
:100120001AE0109370001FEF10936F00F0926B00B5
:1001300017E03122EAE3F1E08894EE1FFF1FE30DA0
:10014000FF1DC89500926C0030916B00230FBB27F8
:10015000A22F3C92339530936B001AE010937000FD
:1001600009C030916B00230FBB27A22F3C921FEFD9
:1001700010936E001F911FBF1F913F902F901F90F3
:10018000FF91EF91BF91AF910F903F912F911895F3
:10019000AF93BF931F931FB71F9310916D001395DB
:1001A00010936D00155041F0A6E610916D00A10F5F
:1001B000BB271C911CB906C053985598F092680053
:1001C000F09269001F911FBF1F91BF91AF911895C9
:1001D00018951FED1DBFFF24A0E6B0E0FD9219EDBC
:1001E0001A1BE1F71FE015BF10EC1BBF18E019BF89
:1001F00012E013BF10E01FBD11E41EBDA89518E06A
:1002000011BD112718BB12BB10E017BB10E011BBCA
:1002100014E91AB91CE019B913E018B92FD0C7D0E6
:10022000FDD020D17894DD24F2BE8CE792B79817E8
:10023000EAF31CE7810FEEE2F1E013E0D122ED2CAE
:100240008894EE1C8894EE1FFF1FEE0DFF1DC895CD
:10025000EEE2F1E0E00DFF1DD394099404000600E6
:1002600008000A0030D0E2CFA3D0E0CFD8D0DECF54
:10027000FAD0DCCF030505010101030277276627C9
:1002800019B71F7B19BF22E03327AEE9B0E01CB3DA
:1002900010FBEEF33EBB11E01CBB1DB31D93339569
:1002A0002A952223A1F716B310FB70F90EF052988D
:1002B00011FB2EF017E619B9F0929F0008951091E6
:1002C0009E0019B9089510906E00112009F46DC0B8
:1002D000F0926E00EBE7F1E0109060008894111C42
:1002E0008894EE1FFF1FE10DFF1DC895EBE7F1E0BD
:1002F000E00DFF1D09940800080008000800080030
:1003000009000A00280050C04FC01091610010FB86
:1003100056F0A0EAB0E010916200A10FBF1D10914D
:1003200063001C9341C01CB311FBEEF310916200FB
:100330001EBB109163001DBBF89414E01CBB12E0BF
:100340001CBB789431C01091610010FBFEF011FBD2
:1003500066F0A0EAB0E010916200A10FBF1DF0921C
:1003600068001C91109369001FC0A0EAB0E01091D2
:100370006200A10FBF1D1D912C913E91311B3323B3
:10038000A1F710936800209369000EC01CB310FB06
:10039000EEF3109162001EBB11E01CBB2DB3F09276
:1003A00068002093690000C07460A89508950895BE
:1003B00077FB0EF031C0579872FB2EF473771091D3
:1003C0009F0010680DC0209170002A952093700046
:1003D00019F573FB77770EF41FC010919F001F77FC
:1003E00076FB16F910936600F0926F00F0926B00A6
:1003F0001091660020916700120F20916800120F83
:1004000020916900120F10936A00F0926D00109114
:100410006600539A1CB9559A579A089508955090BA
:100420007100552009F41DC0A1E3A0535090610054
:10043000A51918F4F092710014C0F0927100E0E375
:10044000F2E0509061008894551C8894EE1FFF1FC5
:10045000E50DFF1DC895E0E3F2E0E00DFF1D0994F6
:1004600001000895089520B336B3221F36953695BE
:1004700036952795369527953695279520907900BE
:1004800030907800222633264090770050907600F6
:1004900060907900709078004624572424283528ED
:1004A000122D1329112399F0422C532C409450946F
:1004B000422253226090A1007090A000622073201D
:1004C000642875286092A1007092A00004C0209357
:1004D000A1003093A0002090770030907600209209
:1004E0007900309278002093770030937600089559
:00000001FF
